:03F0000002F00813
:03F0610002F003B7
:05F0030012F06480FE24
:08F0640090FE00E0FA75E104E2
:0DF06C0090DF3BE0FBBB01F875E1037B008A
:09F079008A047D000CBC00010DAD
:0EF082008B067F00EEB50406EFB50502801286
:05F0900010890280FB65
:0DF095008B040B8C827583FEE0F5D980D7CB
:0AF0A20090DF3BE0FBBB130280F699
:03F0AC0075E10209
:0CF0AF0090DF3BE0FBBB0DF87A107B000B
:09F0BB008A047D000CBC00010D6B
:0EF0C4008B067F00C3EE9CEF64808DF063F03E
:08F0D2008095F0400302F0FC00
:05F0DA0010890280FB1B
:0EF0DF0090DF3BE0FCBC0D118B827583FEE5DB
:0BF0ED00D9FCF00B90FE00E0FA80C39D
:04F0F800A502F0BBC2
:05F0FC0075E104A522EE
:06F03700E478FFF6D8FDAD
:08F015007900E94400601B7A58
:05F01D000090F10578F0
:03F02200007593E3
:0AF0250000E493F2A308B80002050E
:08F02F0093D9F4DAF27593FFA6
:08F03D007800E84400600A7944
:03F04500007593C0
:06F0480000E4F309D8FC0E
:08F04E007800E84400600C7931
:0BF0560000900000E4F0A3D8FCD9FA01
:03F0080075810708
:0AF00B0012F101E582600302F00338
:04F1010075820022F1
:00000001FF
